:10000000D028FF3FFF3FFF3FFF00030E8301B600F4
:100010000408B5000A08B7008A017008B900850114
:100020008701860120088316850083122108831624
:1000300087008312220886002F08233F84000008CF
:10004000A200301C2628F030A20528280F30A20577
:1000500005302F0203185228BF30A1002F08003AA4
:10006000031D35283D30A00086282F08013A031DC6
:100070003C283B30A00086282F08023A031D432865
:100080003730A00086282F08033A031D4A282F3056
:10009000A00086282F08043A031D51281F30A00015
:1000A000862886283F30A0002F08053A031D5B28CC
:1000B000BE30A10086282F08063A031D6228BD30F5
:1000C000A10086282F08073A031D6928BB30A1002C
:1000D00086282F08083A031D7028B730A10086280B
:1000E0002F08093A031D7728AF30A10086282F0872
:1000F0000A3A031D7E289F30A10086282F080B3A5C
:10010000031D86283E30A000BF30A100AF0A0C308E
:100110002F02031C8D28AF01B00A0B113908F00023
:1001200037088A0035088400360E8300FF0E7F0EE4
:100130000900031383123808803A031DB2283108DE
:10014000233FF100710884000008F0007017710867
:10015000840070088000B10A31080B3C0318B128F4
:10016000B101CF28B201381CB628B216B81CB92884
:10017000B214381DBC28B217B81DBF28B215381EDE
:10018000C2283216B81EC5283214381FC8283215A6
:100190003108233FF0007008840032088000080016
:1001A000031383129F01073083169F00831285017A
:1001B00083168501831286018316860183128701C7
:1001C0008030831687008B018930810001308312D3
:1001D00090009201AF01B1014030B8009920013088
:1001E000B1006D30B80099200230B1007930B8000C
:1001F00099200330B1005030B80099200430B1008C
:100200000430B80099200530B1007730B80099204B
:100210000630B1003830B80099200730B100B8017D
:1002200099200830B1001C30B80099200930B10085
:100230000630B80099200930B1008030B80099200C
:100240000A30B1003F30B80099200B30B100403087
:10025000B8009920A0308B001E30B3008F01330806
:10026000031937290C1C36290C10B3032F298316C8
:100270008C0104309800333099009030831298003C
:100280001A08B4001A08B400B10100308C1A013009
:10029000F1007108013A031D6B298F011A08B4009F
:1002A000B41F62290F303405F1007108B1007108E4
:1002B0000B3C03185C29B101341F61298030B80060
:1002C00099206B293408B8009920B10A31080B3CF9
:1002D00003186B29B1019C300F02031C84298F0184
:1002E000003098180130F1007108031D7E2900309C
:1002F00018190130F1007108031984291A08B40093
:100300001A08B4001812181645298529FF3FFF3F27
:02400E00723FFF
:00000001FF
